:1000000019C018951895189518951895189518955C
:100010001895189518951895189518951895189578
:100020001895189518951895189518951895189568
:10003000189518958FEF8DBFC0EEE8ED4E2E82E03B
:100040008EBFD2E0F2E05F2EEEEFF1E0A0E0B1E093
:10005000A89584B7082E877F84BF88E1992780936D
:1000600060009093600088278D933197E9F76624AC
:100070003B983A98529853985498219A229A81EA38
:100080008093800081E0809381003D9A45983C9A5E
:100090003B9A5398549888E592E0A4E0B1E08D93A0
:1000A0009C9380E090E0A0E0B1E08D939C9384E18C
:1000B00090E0A2E0B1E08D939C9380E090E090937B
:1000C0008B0080938A008FEF90E09093890080935B
:1000D000880084EF91E082D0449A439884EF91E0C5
:1000E0007DD04498439A84EF91E078D04498439827
:1000F000A0E0B1E00D911C9141E050E0040F151F0C
:10010000A0E0B1E00D931C93A2E0B1E00D911C9131
:1001100048E250E0040F151FA2E0B1E00D931C93DC
:10012000A2E0B1E08D919C9190938B0080938A0026
:1001300088EC90E053D0A0E0B1E00D911C91053027
:1001400050E0150709F0D4CF80E090E090938B0049
:1001500080938A000027A9E2B0E08C9183FB0EF423
:1001600001E041E0041709F007C080E090E09093BF
:1001700089008093880006C08DEF90E090938900FD
:10018000809388000027A9E2B0E08C9184FB0EF4F4
:1001900001E041E0041709F007C084EB90E0909380
:1001A0008B0080938A0006C084EF90E090938B00D0
:1001B00080938A0001D0CECF439A84E690E00ED09F
:1001C000439884E690E00AD008953197F1F70895B6
:1001D000689462F80895E89462F80895EF93FF93A5
:1001E000EE27E82BE92B31F0E0EDF7E03197F1F75E
:0A01F0000197D1F7FF91EF910895F8
:00000001FF
